BL51 BANKED LINKER/LOCATER V6.05                                                        03/08/2012  15:48:59  PAGE 1


BL51 BANKED LINKER/LOCATER V6.05, INVOKED BY:
C:\KEIL\C51\BIN\BL51.EXE STARTUP.obj, EKTC52C .obj TO EKTC52C RAMSIZE (256) CODE (0X0000-0X3FFF)


MEMORY MODEL: LARGE


INPUT MODULES INCLUDED:
  STARTUP.obj (?C_STARTUP)
  EKTC52C .obj (EKTC52C_)
  C:\KEIL\C51\LIB\C51L.LIB (?C_INIT)
  C:\KEIL\C51\LIB\C51L.LIB (?C?CLDPTR)
  C:\KEIL\C51\LIB\C51L.LIB (?C?CLDOPTR)
  C:\KEIL\C51\LIB\C51L.LIB (?C?IMUL)
  C:\KEIL\C51\LIB\C51L.LIB (?C?UIDIV)
  C:\KEIL\C51\LIB\C51L.LIB (?C?LMUL)
  C:\KEIL\C51\LIB\C51L.LIB (?C?ULDIV)
  C:\KEIL\C51\LIB\C51L.LIB (?C?LSTXDATA)
  C:\KEIL\C51\LIB\C51L.LIB (?C?LSTKXDATA)


LINK MAP OF MODULE:  EKTC52C (?C_STARTUP)


            TYPE    BASE      LENGTH    RELOCATION   SEGMENT NAME
            -----------------------------------------------------

            * * * * * * *   D A T A   M E M O R Y   * * * * * * *
            REG     0000H     0008H     ABSOLUTE     "REG BANK 0"
                    0008H     0018H                  *** GAP ***
            BIT     0020H.0   0002H.1   UNIT         ?BI?EKTC52C_
                    0022H.1   0000H.7                *** GAP ***
            IDATA   0023H     0001H     UNIT         ?STACK

            * * * * * * *  X D A T A   M E M O R Y  * * * * * * *
            XDATA   0000H     01F6H     UNIT         ?XD?EKTC52C_
            XDATA   01F6H     0003H     UNIT         _XDATA_GROUP_

            * * * * * * *   C O D E   M E M O R Y   * * * * * * *
            CODE    0000H     0003H     ABSOLUTE     
                    0003H     0008H                  *** GAP ***
            CODE    000BH     0003H     ABSOLUTE     
            CODE    000EH     0014H     UNIT         ?PR?_PIC_STR?EKTC52C_
                    0022H     0001H                  *** GAP ***
            CODE    0023H     0003H     ABSOLUTE     
            CODE    0026H     0733H     UNIT         ?PR?MAIN?EKTC52C_
            CODE    0759H     0207H     UNIT         ?C?LIB_CODE
            CODE    0960H     0206H     UNIT         ?PR?_CHECK?EKTC52C_
            CODE    0B66H     0202H     UNIT         ?CO?EKTC52C_
            CODE    0D68H     01B1H     UNIT         ?C_INITSEG
            CODE    0F19H     013CH     UNIT         ?PR?SYS_INIT?EKTC52C_
            CODE    1055H     00D3H     UNIT         ?PR?_PRINTF?EKTC52C_
            CODE    1128H     009DH     UNIT         ?PR?UART_ISR?EKTC52C_
            CODE    11C5H     0093H     UNIT         ?PR?TIMER0?EKTC52C_
            CODE    1258H     008CH     UNIT         ?C_C51STARTUP
            CODE    12E4H     0072H     UNIT         ?PR?_HEXDSP?EKTC52C_
            CODE    1356H     0057H     UNIT         ?PR?_WRXRAM?EKTC52C_
            CODE    13ADH     0050H     UNIT         ?PR?_HWTST_71?EKTC52C_
BL51 BANKED LINKER/LOCATER V6.05                                                      03/08/2012  15:48:59  PAGE 2


            CODE    13FDH     0039H     UNIT         ?PR?_UART_TRANSMIT?EKTC52C_
            CODE    1436H     001CH     UNIT         ?PR?_DSP?EKTC52C_
            CODE    1452H     001BH     UNIT         ?PR?_SEND_STR?EKTC52C_
            CODE    146DH     0018H     UNIT         ?PR?_DELAY?EKTC52C_
            CODE    1485H     000DH     UNIT         ?PR?EN?EKTC52C_



OVERLAY MAP OF MODULE:   EKTC52C (?C_STARTUP)


SEGMENT                               XDATA_GROUP
  +--> CALLED SEGMENT               START    LENGTH
---------------------------------------------------
?C_C51STARTUP                       -----    -----
  +--> ?PR?MAIN?EKTC52C_
  +--> ?C_INITSEG

?PR?MAIN?EKTC52C_                   -----    -----
  +--> ?PR?SYS_INIT?EKTC52C_
  +--> ?PR?_DELAY?EKTC52C_
  +--> ?PR?EN?EKTC52C_
  +--> ?PR?_SEND_STR?EKTC52C_
  +--> ?PR?_UART_TRANSMIT?EKTC52C_
  +--> ?PR?_HEXDSP?EKTC52C_
  +--> ?PR?_CHECK?EKTC52C_
  +--> ?PR?_PIC_STR?EKTC52C_
  +--> ?PR?_DSP?EKTC52C_
  +--> ?PR?_HWTST_71?EKTC52C_
  +--> ?PR?_WRXRAM?EKTC52C_
  +--> ?PR?_PRINTF?EKTC52C_

?PR?EN?EKTC52C_                     -----    -----
  +--> ?PR?_UART_TRANSMIT?EKTC52C_
  +--> ?PR?_SEND_STR?EKTC52C_

?PR?_SEND_STR?EKTC52C_              -----    -----
  +--> ?PR?_UART_TRANSMIT?EKTC52C_

?PR?_HEXDSP?EKTC52C_                -----    -----
  +--> ?PR?_UART_TRANSMIT?EKTC52C_
  +--> ?PR?_SEND_STR?EKTC52C_

?PR?_CHECK?EKTC52C_                 01F6H    0002H
  +--> ?CO?EKTC52C_

?PR?_PIC_STR?EKTC52C_               -----    -----
  +--> ?PR?_UART_TRANSMIT?EKTC52C_
  +--> ?PR?EN?EKTC52C_

?PR?_DSP?EKTC52C_                   -----    -----
  +--> ?PR?_SEND_STR?EKTC52C_
  +--> ?PR?_UART_TRANSMIT?EKTC52C_

?PR?_HWTST_71?EKTC52C_              -----    -----
  +--> ?PR?_UART_TRANSMIT?EKTC52C_
  +--> ?PR?EN?EKTC52C_
BL51 BANKED LINKER/LOCATER V6.05                                                      03/08/2012  15:48:59  PAGE 3



?PR?_PRINTF?EKTC52C_                01F6H    0003H
  +--> ?PR?_SEND_STR?EKTC52C_
  +--> ?CO?EKTC52C_
  +--> ?PR?_UART_TRANSMIT?EKTC52C_



UNRESOLVED EXTERNAL SYMBOLS:
   KEY



SYMBOL TABLE OF MODULE:  EKTC52C (?C_STARTUP)

  VALUE           TYPE          NAME
  ----------------------------------

  -------         MODULE        ?C_STARTUP
  C:1258H         SEGMENT       ?C_C51STARTUP
  I:0023H         SEGMENT       ?STACK
  C:0000H         PUBLIC        ?C_STARTUP
  D:00E0H         SYMBOL        ACC
  D:00F0H         SYMBOL        B
  D:0083H         SYMBOL        DPH
  D:0082H         SYMBOL        DPL
  N:0000H         SYMBOL        IBPSTACK
  N:0100H         SYMBOL        IBPSTACKTOP
  N:0080H         SYMBOL        IDATALEN
  C:125BH         SYMBOL        IDATALOOP
  N:0000H         SYMBOL        PBPSTACK
  N:0100H         SYMBOL        PBPSTACKTOP
  N:0000H         SYMBOL        PDATALEN
  N:0000H         SYMBOL        PDATASTART
  N:0000H         SYMBOL        PPAGE
  N:0000H         SYMBOL        PPAGEENABLE
  D:00A0H         SYMBOL        PPAGE_SFR
  D:0081H         SYMBOL        SP
  C:1258H         SYMBOL        STARTUP1
  N:0000H         SYMBOL        XBPSTACK
  N:0000H         SYMBOL        XBPSTACKTOP
  N:0000H         SYMBOL        XDATALEN
  N:0000H         SYMBOL        XDATASTART
  C:0000H         LINE#         126
  C:1258H         LINE#         133
  C:125AH         LINE#         134
  C:125BH         LINE#         135
  C:125CH         LINE#         136
  C:125EH         LINE#         185
  C:1261H         LINE#         196
  -------         ENDMOD        ?C_STARTUP

  -------         MODULE        EKTC52C_
  C:0000H         SYMBOL        _ICE_DUMMY_
  D:0080H         PUBLIC        P0
  X:0000H         PUBLIC        CMD7C1
  D:0090H         PUBLIC        P1
BL51 BANKED LINKER/LOCATER V6.05                                                      03/08/2012  15:48:59  PAGE 4


  X:0017H         PUBLIC        CMD7C2
  X:002CH         PUBLIC        RTC250
  D:00B0H         PUBLIC        P3
  B:0020H.0       PUBLIC        RTCOK
  X:002EH         PUBLIC        RTC128
  B:00A8H.7       PUBLIC        EA
  B:0020H.1       PUBLIC        LED1
  X:0030H         PUBLIC        RTCON
  B:0020H.2       PUBLIC        LED2
  X:0040H         PUBLIC        HRNUM
  C:1128H         PUBLIC        UART_ISR
  X:0041H         PUBLIC        HRPOS
  X:0053H         PUBLIC        dattmp
  D:00A8H         PUBLIC        IE
  B:0020H.3       PUBLIC        JDQ1
  C:146DH         PUBLIC        _delay
  B:0020H.4       PUBLIC        JDQ2
  B:0020H.5       PUBLIC        JDQ3
  B:0020H.6       PUBLIC        JDQ4
  C:1055H         PUBLIC        _printf
  B:00A8H.4       PUBLIC        ES
  D:00B8H         PUBLIC        IP
  B:0020H.7       PUBLIC        KEY1
  B:0098H.0       PUBLIC        RI
  C:0B66H         PUBLIC        ZB
  B:0021H.0       PUBLIC        KEY2
  B:0098H.1       PUBLIC        TI
  X:0054H         PUBLIC        QQ
  X:0055H         PUBLIC        CMD7CT
  C:0026H         PUBLIC        main
  X:007CH         PUBLIC        ADNUM0
  X:007EH         PUBLIC        ADNUM1
  X:0080H         PUBLIC        TT
  X:0081H         PUBLIC        ADNUM2
  X:0083H         PUBLIC        ADNUM3
  X:0085H         PUBLIC        ADNUM4
  X:0087H         PUBLIC        Tim
  X:0089H         PUBLIC        Tjm
  B:0021H.1       PUBLIC        RXFRMOK
  D:0099H         PUBLIC        SBUF
  D:0087H         PUBLIC        PCON
  C:11C5H         PUBLIC        Timer0
  X:008BH         PUBLIC        ZZ
  D:0098H         PUBLIC        SCON
  X:008DH         PUBLIC        AD0
  X:0091H         PUBLIC        DNUM
  D:0089H         PUBLIC        TMOD
  D:0088H         PUBLIC        TCON
  X:0092H         PUBLIC        AD1
  X:0096H         PUBLIC        AD2
  X:009AH         PUBLIC        AD_R
  B:0080H.0       PUBLIC        LED01
  X:009CH         PUBLIC        AD3
  B:0080H.1       PUBLIC        LED02
  X:00A0H         PUBLIC        CMD40
  X:00ABH         PUBLIC        AD4
  X:00AFH         PUBLIC        dat
BL51 BANKED LINKER/LOCATER V6.05                                                      03/08/2012  15:48:59  PAGE 5


  X:00DFH         PUBLIC        rec
  X:00F9H         PUBLIC        CMD70
  X:010BH         PUBLIC        CMD71
  X:011FH         PUBLIC        CMD55
  X:0126H         PUBLIC        RTCCEN
  X:012FH         PUBLIC        PNUM
  B:0080H.2       PUBLIC        JDQ01
  B:0080H.3       PUBLIC        JDQ02
  B:0080H.4       PUBLIC        JDQ03
  B:0080H.5       PUBLIC        JDQ04
  X:0130H         PUBLIC        TNUM
  B:0021H.2       PUBLIC        RXAAOK
  X:0131H         PUBLIC        CMDD0
  X:0138H         PUBLIC        WINFLG
  B:00A8H.1       PUBLIC        ET0
  X:0139H         PUBLIC        CMDTTL
  X:013EH         PUBLIC        CMDE0
  X:014DH         PUBLIC        RTCOLD
  B:0088H.5       PUBLIC        TF0
  D:008CH         PUBLIC        TH0
  X:014EH         PUBLIC        SECNUM
  D:008DH         PUBLIC        TH1
  C:12E9H         PUBLIC        _HEXDSP
  X:014FH         PUBLIC        SECPOS
  X:0161H         PUBLIC        CMD9B
  B:0021H.3       PUBLIC        AD0OK
  D:008AH         PUBLIC        TL0
  X:0169H         PUBLIC        CMDE7
  B:0021H.4       PUBLIC        AD1OK
  D:008BH         PUBLIC        TL1
  B:0021H.5       PUBLIC        AD2OK
  C:1489H         PUBLIC        en
  B:0021H.6       PUBLIC        AD3OK
  B:0021H.7       PUBLIC        AD4OK
  X:0170H         PUBLIC        MINNUM
  B:0088H.4       PUBLIC        TR0
  B:0088H.6       PUBLIC        TR1
  X:0171H         PUBLIC        MINPOS
  X:0183H         PUBLIC        DSPNUM
  X:0184H         PUBLIC        ADT
  C:0960H         PUBLIC        _CHECK
  X:0185H         PUBLIC        LEN
  X:0186H         PUBLIC        CMD71TP
  C:1356H         PUBLIC        _WRXRAM
  C:13ADH         PUBLIC        _HWTST_71
  C:0B72H         PUBLIC        PT1000
  X:019AH         PUBLIC        CMD7CTB
  X:01AEH         PUBLIC        ADTIME0
  C:1436H         PUBLIC        _DSP
  C:1458H         PUBLIC        _send_str
  X:01AFH         PUBLIC        TMPNOW
  X:01B1H         PUBLIC        ADTIME1
  D:00C8H         PUBLIC        T2CON
  X:01B2H         PUBLIC        ADTIME2
  X:01B4H         PUBLIC        i
  X:01B5H         PUBLIC        ADTIME3
  X:01B6H         PUBLIC        j
BL51 BANKED LINKER/LOCATER V6.05                                                      03/08/2012  15:48:59  PAGE 6


  B:0022H.0       PUBLIC        TI0FLAG
  X:01B7H         PUBLIC        k
  X:01B9H         PUBLIC        ADTIME4
  X:01BAH         PUBLIC        CMD551
  C:0F19H         PUBLIC        SYS_Init
  C:142CH         PUBLIC        _Uart_transmit
  X:01BDH         PUBLIC        CMD981
  C:000EH         PUBLIC        _pic_str
  X:01CBH         PUBLIC        CMD982
  X:01D9H         PUBLIC        CMD983
  X:01E7H         PUBLIC        T_F
  X:01E8H         PUBLIC        CMD984
  D:00D0H         PUBLIC        PSW
  -------         PROC          L?0184
  -------         ENDPROC       L?0184
  -------         PROC          _UART_TRANSMIT
  D:0007H         SYMBOL        i
  C:142CH         LINE#         175
  C:142CH         LINE#         176
  C:142CH         LINE#         177
  C:142EH         LINE#         178
  C:1430H         LINE#         179
  C:1433H         LINE#         180
  C:1435H         LINE#         181
  -------         ENDPROC       _UART_TRANSMIT
  C:1452H         SYMBOL        L?0186
  -------         PROC          L?0185
  -------         ENDPROC       L?0185
  C:1452H         SYMBOL        L?0186
  -------         PROC          _SEND_STR
  D:0001H         SYMBOL        p
  C:1458H         LINE#         184
  C:1458H         LINE#         185
  C:1458H         LINE#         186
  C:1460H         LINE#         187
  C:1460H         LINE#         188
  C:1463H         LINE#         189
  C:146CH         LINE#         190
  -------         ENDPROC       _SEND_STR
  -------         PROC          UART_ISR
  -------         DO            
  D:0007H         SYMBOL        i
  -------         ENDDO         
  C:1128H         LINE#         196
  C:1137H         LINE#         200
  C:113AH         LINE#         201
  C:113AH         LINE#         202
  C:113CH         LINE#         203
  C:113EH         LINE#         205
  C:1141H         LINE#         206
  C:1141H         LINE#         207
  C:1144H         LINE#         208
  C:1144H         LINE#         209
  C:1153H         LINE#         210
  C:1159H         LINE#         211
  C:1160H         LINE#         212
  C:1160H         LINE#         213
BL51 BANKED LINKER/LOCATER V6.05                                                      03/08/2012  15:48:59  PAGE 7


  C:11A1H         LINE#         214
  C:11A1H         LINE#         215
  C:11A3H         LINE#         216
  C:11A5H         LINE#         217
  C:11A5H         LINE#         218
  C:11A5H         LINE#         219
  C:11A7H         LINE#         221
  C:11A7H         LINE#         222
  C:11ABH         LINE#         223
  C:11ABH         LINE#         224
  C:11ADH         LINE#         225
  C:11B2H         LINE#         226
  C:11B2H         LINE#         227
  C:11B2H         LINE#         228
  C:11B2H         LINE#         229
  C:11B4H         LINE#         231
  C:11B4H         LINE#         232
  C:11B6H         LINE#         233
  C:11B8H         LINE#         234
  C:11B8H         LINE#         235
  -------         ENDPROC       UART_ISR
  -------         PROC          TIMER0
  C:11C5H         LINE#         240
  C:11CDH         LINE#         242
  C:11CFH         LINE#         243
  C:11D1H         LINE#         244
  C:11D4H         LINE#         245
  C:11D7H         LINE#         246
  C:11E5H         LINE#         247
  C:11F4H         LINE#         248
  C:11F4H         LINE#         249
  C:11F8H         LINE#         250
  C:11FAH         LINE#         251
  C:11FAH         LINE#         252
  C:1215H         LINE#         253
  C:1217H         LINE#         255
  C:1225H         LINE#         256
  C:123AH         LINE#         269
  C:1246H         LINE#         270
  C:1246H         LINE#         271
  C:124DH         LINE#         272
  C:124FH         LINE#         273
  C:124FH         LINE#         275
  -------         ENDPROC       TIMER0
  -------         PROC          _DELAY
  D:0006H         SYMBOL        x
  C:146DH         LINE#         313
  C:146DH         LINE#         314
  C:146DH         LINE#         319
  C:147AH         LINE#         320
  C:1484H         LINE#         321
  -------         ENDPROC       _DELAY
  C:1485H         SYMBOL        L?0190
  -------         PROC          L?0189
  -------         ENDPROC       L?0189
  C:1485H         SYMBOL        L?0190
  -------         PROC          EN
BL51 BANKED LINKER/LOCATER V6.05                                                      03/08/2012  15:48:59  PAGE 8


  C:1489H         LINE#         326
  C:1489H         LINE#         327
  C:1489H         LINE#         328
  -------         ENDPROC       EN
  -------         PROC          _PIC_STR
  D:0006H         SYMBOL        i
  C:000EH         LINE#         334
  C:0010H         LINE#         335
  C:0010H         LINE#         336
  C:0015H         LINE#         337
  C:001AH         LINE#         338
  C:001FH         LINE#         339
  -------         ENDPROC       _PIC_STR
  -------         PROC          _WRXRAM
  D:0007H         SYMBOL        n
  D:0001H         SYMBOL        p
  C:1356H         LINE#         345
  C:1356H         LINE#         346
  C:1356H         LINE#         347
  C:1365H         LINE#         348
  C:1365H         LINE#         349
  C:136AH         LINE#         350
  C:136AH         LINE#         351
  C:138CH         LINE#         352
  C:138EH         LINE#         353
  C:13A4H         LINE#         354
  C:13ACH         LINE#         355
  -------         ENDPROC       _WRXRAM
  C:12E4H         SYMBOL        L?0188
  -------         PROC          L?0187
  -------         ENDPROC       L?0187
  C:12E4H         SYMBOL        L?0188
  -------         PROC          _HEXDSP
  D:0002H         SYMBOL        num
  C:12E9H         LINE#         360
  C:12EDH         LINE#         361
  C:12EDH         LINE#         362
  C:12F9H         LINE#         363
  C:1309H         LINE#         364
  C:1313H         LINE#         365
  C:131FH         LINE#         366
  C:132DH         LINE#         367
  C:1338H         LINE#         368
  C:133FH         LINE#         369
  C:1346H         LINE#         370
  C:134FH         LINE#         372
  -------         ENDPROC       _HEXDSP
  -------         PROC          _DSP
  D:0006H         SYMBOL        i
  D:0005H         SYMBOL        j
  C:1436H         LINE#         378
  C:1438H         LINE#         379
  C:1438H         LINE#         380
  C:1441H         LINE#         381
  C:1446H         LINE#         382
  C:144BH         LINE#         383
  -------         ENDPROC       _DSP
BL51 BANKED LINKER/LOCATER V6.05                                                      03/08/2012  15:48:59  PAGE 9


  -------         PROC          _PRINTF
  X:01F6H         SYMBOL        p
  C:1055H         LINE#         389
  C:1060H         LINE#         390
  C:1060H         LINE#         391
  C:1065H         LINE#         392
  C:1065H         LINE#         393
  C:1068H         LINE#         395
  C:107FH         LINE#         396
  C:1097H         LINE#         397
  C:10AEH         LINE#         398
  C:10C6H         LINE#         400
  C:10DDH         LINE#         401
  C:110FH         LINE#         402
  C:1118H         LINE#         403
  C:1127H         LINE#         404
  -------         ENDPROC       _PRINTF
  -------         PROC          _HWTST_71
  D:0006H         SYMBOL        i
  D:0004H         SYMBOL        j
  D:0002H         SYMBOL        k
  C:13ADH         LINE#         409
  C:13AFH         LINE#         410
  C:13AFH         LINE#         411
  C:13B4H         LINE#         412
  C:13B9H         LINE#         413
  C:13BEH         LINE#         414
  C:13D2H         LINE#         415
  C:13E6H         LINE#         416
  C:13FAH         LINE#         417
  -------         ENDPROC       _HWTST_71
  -------         PROC          _CHECK
  X:01F6H         SYMBOL        i
  -------         DO            
  X:01F7H         SYMBOL        j
  -------         ENDDO         
  C:0960H         LINE#         453
  C:0965H         LINE#         454
  C:0965H         LINE#         457
  C:096AH         LINE#         458
  C:096AH         LINE#         459
  C:0979H         LINE#         460
  C:0979H         LINE#         461
  C:099EH         LINE#         462
  C:099EH         LINE#         463
  C:09BAH         LINE#         465
  C:09BAH         LINE#         466
  C:09DBH         LINE#         467
  C:09DBH         LINE#         468
  C:0A43H         LINE#         469
  C:0A53H         LINE#         471
  C:0A53H         LINE#         472
  C:0A5CH         LINE#         473
  C:0A5CH         LINE#         474
  C:0A67H         LINE#         475
  C:0A67H         LINE#         476
  C:0A76H         LINE#         477
BL51 BANKED LINKER/LOCATER V6.05                                                      03/08/2012  15:48:59  PAGE 10


  C:0A76H         LINE#         478
  C:0A9DH         LINE#         479
  C:0A9DH         LINE#         480
  C:0AB0H         LINE#         482
  C:0AB0H         LINE#         483
  C:0AD6H         LINE#         484
  C:0AD6H         LINE#         485
  C:0B3DH         LINE#         486
  C:0B5CH         LINE#         488
  C:0B5CH         LINE#         489
  C:0B65H         LINE#         490
  C:0B65H         LINE#         491
  -------         ENDPROC       _CHECK
  -------         PROC          SYS_INIT
  C:0F19H         LINE#         496
  C:0F19H         LINE#         497
  C:0F19H         LINE#         498
  C:0F1CH         LINE#         499
  C:0F1FH         LINE#         500
  C:0F22H         LINE#         501
  C:0F25H         LINE#         502
  C:0F28H         LINE#         503
  C:0F2AH         LINE#         504
  C:0F2CH         LINE#         505
  C:0F2FH         LINE#         506
  C:0F32H         LINE#         507
  C:0F34H         LINE#         508
  C:0F36H         LINE#         510
  C:0F50H         LINE#         511
  C:0F52H         LINE#         512
  C:0F54H         LINE#         513
  C:0F86H         LINE#         514
  C:0F8BH         LINE#         515
  C:0F8FH         LINE#         516
  C:0F93H         LINE#         517
  C:0F99H         LINE#         518
  C:0F9EH         LINE#         519
  C:0FBAH         LINE#         520
  C:0FC4H         LINE#         521
  C:0FCEH         LINE#         522
  C:0FDEH         LINE#         523
  C:0FF4H         LINE#         524
  C:0FF8H         LINE#         525
  C:0FFEH         LINE#         526
  C:1014H         LINE#         527
  C:1031H         LINE#         528
  C:1040H         LINE#         529
  C:1054H         LINE#         530
  -------         ENDPROC       SYS_INIT
  -------         PROC          MAIN
  C:0026H         LINE#         535
  C:0026H         LINE#         536
  C:0026H         LINE#         537
  C:0028H         LINE#         538
  C:002BH         LINE#         539
  C:002DH         LINE#         540
  C:0034H         LINE#         542
BL51 BANKED LINKER/LOCATER V6.05                                                      03/08/2012  15:48:59  PAGE 11


  C:0037H         LINE#         543
  C:0040H         LINE#         544
  C:0047H         LINE#         545
  C:004CH         LINE#         546
  C:0051H         LINE#         547
  C:0052H         LINE#         548
  C:0055H         LINE#         549
  C:005EH         LINE#         550
  C:0063H         LINE#         552
  C:0063H         LINE#         553
  C:0063H         LINE#         554
  C:0066H         LINE#         556
  C:0071H         LINE#         557
  C:0071H         LINE#         558
  C:0074H         LINE#         559
  C:0074H         LINE#         560
  C:0076H         LINE#         561
  C:007CH         LINE#         562
  C:0084H         LINE#         563
  C:0084H         LINE#         564
  C:00A2H         LINE#         565
  C:00B1H         LINE#         566
  C:00B4H         LINE#         567
  C:00B9H         LINE#         568
  C:00BEH         LINE#         569
  C:00C3H         LINE#         570
  C:00C8H         LINE#         571
  C:00CEH         LINE#         573
  C:00DCH         LINE#         574
  C:00DCH         LINE#         575
  C:00DFH         LINE#         576
  C:00E2H         LINE#         577
  C:00E2H         LINE#         578
  C:00E4H         LINE#         579
  C:00EAH         LINE#         580
  C:00F2H         LINE#         581
  C:00F2H         LINE#         582
  C:0111H         LINE#         583
  C:0120H         LINE#         584
  C:0123H         LINE#         585
  C:0128H         LINE#         586
  C:012DH         LINE#         587
  C:0132H         LINE#         588
  C:0137H         LINE#         589
  C:013DH         LINE#         591
  C:014BH         LINE#         592
  C:014BH         LINE#         593
  C:014EH         LINE#         594
  C:0154H         LINE#         595
  C:0154H         LINE#         596
  C:0156H         LINE#         597
  C:0164H         LINE#         598
  C:0173H         LINE#         599
  C:0173H         LINE#         600
  C:0190H         LINE#         601
  C:01D1H         LINE#         602
  C:01E5H         LINE#         603
BL51 BANKED LINKER/LOCATER V6.05                                                      03/08/2012  15:48:59  PAGE 12


  C:0201H         LINE#         604
  C:021FH         LINE#         605
  C:0241H         LINE#         607
  C:0251H         LINE#         608
  C:0251H         LINE#         609
  C:0253H         LINE#         610
  C:0256H         LINE#         611
  C:0256H         LINE#         612
  C:0258H         LINE#         613
  C:025EH         LINE#         614
  C:0263H         LINE#         615
  C:0263H         LINE#         616
  C:0281H         LINE#         617
  C:0284H         LINE#         618
  C:0289H         LINE#         619
  C:028EH         LINE#         620
  C:0293H         LINE#         621
  C:0298H         LINE#         622
  C:029EH         LINE#         624
  C:02B3H         LINE#         625
  C:02B3H         LINE#         626
  C:02B3H         LINE#         646
  C:02B3H         LINE#         648
  C:02B9H         LINE#         649
  C:02B9H         LINE#         650
  C:02BBH         LINE#         652
  C:02C2H         LINE#         653
  C:02C2H         LINE#         654
  C:02CBH         LINE#         655
  C:02D5H         LINE#         656
  C:02DBH         LINE#         657
  C:02DEH         LINE#         658
  C:02E6H         LINE#         659
  C:02E6H         LINE#         660
  C:02EFH         LINE#         661
  C:02F2H         LINE#         662
  C:02F7H         LINE#         663
  C:02F7H         LINE#         664
  C:02FDH         LINE#         665
  C:0305H         LINE#         666
  C:0305H         LINE#         667
  C:0306H         LINE#         668
  C:030EH         LINE#         669
  C:0314H         LINE#         670
  C:031FH         LINE#         671
  C:031FH         LINE#         672
  C:0322H         LINE#         673
  C:032DH         LINE#         674
  C:032DH         LINE#         675
  C:0336H         LINE#         676
  C:0341H         LINE#         677
  C:0360H         LINE#         678
  C:0383H         LINE#         679
  C:03A6H         LINE#         680
  C:03ABH         LINE#         681
  C:03BDH         LINE#         682
  C:03C0H         LINE#         683
BL51 BANKED LINKER/LOCATER V6.05                                                      03/08/2012  15:48:59  PAGE 13


  C:03C0H         LINE#         684
  C:03C0H         LINE#         686
  C:03C6H         LINE#         687
  C:03C6H         LINE#         688
  C:03C8H         LINE#         689
  C:03D3H         LINE#         690
  C:03D3H         LINE#         691
  C:03DBH         LINE#         692
  C:03DBH         LINE#         693
  C:03DDH         LINE#         694
  C:03F4H         LINE#         695
  C:040CH         LINE#         696
  C:041DH         LINE#         697
  C:042DH         LINE#         698
  C:0439H         LINE#         699
  C:0441H         LINE#         700
  C:0445H         LINE#         701
  C:0448H         LINE#         702
  C:0459H         LINE#         703
  C:045CH         LINE#         705
  C:0461H         LINE#         706
  C:0461H         LINE#         707
  C:0473H         LINE#         708
  C:047EH         LINE#         709
  C:047EH         LINE#         710
  C:0482H         LINE#         711
  C:0484H         LINE#         712
  C:0489H         LINE#         713
  C:048EH         LINE#         714
  C:048EH         LINE#         715
  C:0491H         LINE#         716
  C:0496H         LINE#         717
  C:0496H         LINE#         718
  C:0499H         LINE#         719
  C:04A4H         LINE#         720
  C:04A4H         LINE#         721
  C:04AAH         LINE#         722
  C:04AAH         LINE#         723
  C:04B9H         LINE#         724
  C:04C8H         LINE#         725
  C:04CDH         LINE#         726
  C:04D0H         LINE#         727
  C:04D8H         LINE#         728
  C:04D8H         LINE#         729
  C:04E7H         LINE#         730
  C:04F6H         LINE#         731
  C:04FBH         LINE#         732
  C:04FEH         LINE#         735
  C:0506H         LINE#         736
  C:0506H         LINE#         737
  C:0517H         LINE#         738
  C:0526H         LINE#         739
  C:052BH         LINE#         740
  C:052EH         LINE#         741
  C:0536H         LINE#         742
  C:0536H         LINE#         743
  C:0547H         LINE#         744
BL51 BANKED LINKER/LOCATER V6.05                                                      03/08/2012  15:48:59  PAGE 14


  C:0556H         LINE#         745
  C:055BH         LINE#         746
  C:055EH         LINE#         747
  C:0566H         LINE#         748
  C:0566H         LINE#         749
  C:0577H         LINE#         750
  C:0586H         LINE#         751
  C:058BH         LINE#         752
  C:058EH         LINE#         753
  C:0596H         LINE#         754
  C:0596H         LINE#         755
  C:05A7H         LINE#         756
  C:05B6H         LINE#         757
  C:05BBH         LINE#         758
  C:05BEH         LINE#         759
  C:05D3H         LINE#         760
  C:05D3H         LINE#         761
  C:05D6H         LINE#         762
  C:05F0H         LINE#         763
  C:05F0H         LINE#         764
  C:05F2H         LINE#         766
  C:0607H         LINE#         767
  C:061CH         LINE#         768
  C:0630H         LINE#         770
  C:0639H         LINE#         771
  C:0640H         LINE#         772
  C:0657H         LINE#         773
  C:0669H         LINE#         774
  C:0670H         LINE#         776
  C:0682H         LINE#         777
  C:068FH         LINE#         778
  C:069CH         LINE#         779
  C:06A3H         LINE#         780
  C:06ABH         LINE#         781
  C:06B1H         LINE#         782
  C:06B8H         LINE#         784
  C:06BFH         LINE#         785
  C:06CDH         LINE#         786
  C:06D6H         LINE#         787
  C:06DDH         LINE#         789
  C:06E0H         LINE#         790
  C:06EBH         LINE#         791
  C:06EBH         LINE#         792
  C:06F4H         LINE#         793
  C:06F4H         LINE#         794
  C:06FDH         LINE#         795
  C:0709H         LINE#         796
  C:071AH         LINE#         797
  C:0723H         LINE#         798
  C:0726H         LINE#         799
  C:072EH         LINE#         800
  C:072EH         LINE#         801
  C:0737H         LINE#         803
  C:0742H         LINE#         804
  C:0742H         LINE#         805
  C:0749H         LINE#         806
  C:074CH         LINE#         807
BL51 BANKED LINKER/LOCATER V6.05                                                      03/08/2012  15:48:59  PAGE 15


  C:074CH         LINE#         808
  C:074FH         LINE#         809
  C:0750H         LINE#         810
  C:0750H         LINE#         811
  C:0753H         LINE#         812
  C:0756H         LINE#         813
  C:0756H         LINE#         814
  C:0756H         LINE#         815
  C:0756H         LINE#         816
  C:0756H         LINE#         817
  -------         ENDPROC       MAIN
  -------         ENDMOD        EKTC52C_

  -------         MODULE        ?C?CLDPTR
  C:0759H         PUBLIC        ?C?CLDPTR
  -------         ENDMOD        ?C?CLDPTR

  -------         MODULE        ?C?CLDOPTR
  C:0772H         PUBLIC        ?C?CLDOPTR
  -------         ENDMOD        ?C?CLDOPTR

  -------         MODULE        ?C?IMUL
  C:079FH         PUBLIC        ?C?IMUL
  -------         ENDMOD        ?C?IMUL

  -------         MODULE        ?C?UIDIV
  C:07B1H         PUBLIC        ?C?UIDIV
  -------         ENDMOD        ?C?UIDIV

  -------         MODULE        ?C?LMUL
  C:0806H         PUBLIC        ?C?LMUL
  -------         ENDMOD        ?C?LMUL

  -------         MODULE        ?C?ULDIV
  C:0891H         PUBLIC        ?C?ULDIV
  -------         ENDMOD        ?C?ULDIV

  -------         MODULE        ?C?LSTXDATA
  C:0923H         PUBLIC        ?C?LSTXDATA
  -------         ENDMOD        ?C?LSTXDATA

  -------         MODULE        ?C?LSTKXDATA
  C:092FH         PUBLIC        ?C?LSTKXDATA
  -------         ENDMOD        ?C?LSTKXDATA

*** WARNING L1: UNRESOLVED EXTERNAL SYMBOL
    SYMBOL:  KEY
    MODULE:  EKTC52C .obj (EKTC52C_)

*** WARNING L2: REFERENCE MADE TO UNRESOLVED EXTERNAL
    SYMBOL:  KEY
    MODULE:  EKTC52C .obj (EKTC52C_)
    ADDRESS: 0064H

Program Size: data=11.1 xdata=505 code=5257
LINK/LOCATE RUN COMPLETE.  2 WARNING(S),  0 ERROR(S)
